:0FFD6700011300010C00010B00010D00010F0042
:10FBC90012F91512FDBE12FE38E50CB4FF14E51A40
:10FBD900D39400400DD51A0AE47834F67F0AFE1250
:10FBE900FE1B7838E6600712FCF7E47838F620B097
:10FBF900087838E6700312FA387834E6702720B2AC
:10FC090012E50DB4010DD2A3C2A4D2D8C2D9E4F52C
:10FC19000D801220B30FE50D700BD2A3D2A4D2D858
:09FC2900D2D9750D01050C809D76
:10F91500D2A3C2A4D2D8C2D9C2097580FF43BF02FF
:10F925007B007A0079087F007EEE12FE0FAD08E4B9
:10F93500FFFE12FE027B007A0079097F017EEE123E
:10F94500FE0FAD097F017E0012FE027B007A007971
:10F95500147F027EEE12FE0FAD147F027E0012FEB2
:10F96500027B007A0079157F037EEE12FE0FAD153E
:10F975007F037E0012FE027B007A0079127F047EEF
:10F98500EE12FE0FAD127F047E0012FE027B007A9E
:10F995000079107F057EEE12FE0FAD107F057E000B
:10F9A50012FE027B007A00791C7F067EEE12FE0FA6
:10F9B500AD1C7F067E0012FE027B007A0079167F61
:10F9C500077EEE12FE0FAD167F077E0012FE027B4C
:10F9D500007A00790A7F087EEE12FE0FAD0A7F08D5
:10F9E5007E0012FE027B007A00790E7F097EEE1200
:10F9F500FE0FAD0E7F097E0012FE027D207F0B7E7D
:10FA05000012FE027B007A0079117F107EEE12FE55
:10FA15000FAD117F107E0012FE02E5D85408FFE5F8
:10FA2500117006BF08030202007580FBC2B5C2B69D
:03FA3500D2B72223
:04FE3800759FA722E9
:0BFE1B00EF1FAC0670011E4C70F622B9
:10F28C0000C1814001C0804101C0804100C181406A
:10F29C0001C0804100C1814000C1814001C080415A
:10F2AC0001C0804100C1814000C1814001C080414A
:10F2BC0000C1814001C0804101C0804100C181403A
:10F2CC0001C0804100C1814000C1814001C080412A
:10F2DC0000C1814001C0804101C0804100C181401A
:10F2EC0000C1814001C0804101C0804100C181400A
:10F2FC0001C0804100C1814000C1814001C08041FA
:10F30C0001C0804100C1814000C1814001C08041E9
:10F31C0000C1814001C0804101C0804100C18140D9
:10F32C0000C1814001C0804101C0804100C18140C9
:10F33C0001C0804100C1814000C1814001C08041B9
:10F34C0000C1814001C0804101C0804100C18140A9
:10F35C0001C0804100C1814000C1814001C0804199
:10F36C0001C0804100C1814000C1814001C0804189
:10F37C0000C1814001C0804101C0804100C1814079
:10F38C0000C0C101C30302C2C60607C705C5C40439
:10F39C00CC0C0DCD0FCFCE0E0ACACB0BC90908C8A9
:10F3AC00D81819D91BDBDA1A1EDEDF1FDD1D1CDC99
:10F3BC0014D4D515D71716D6D21213D311D1D01009
:10F3CC00F03031F133F3F23236F6F737F53534F4F9
:10F3DC003CFCFD3DFF3F3EFEFA3A3BFB39F9F83869
:10F3EC0028E8E929EB2B2AEAEE2E2FEF2DEDEC2C59
:10F3FC00E42425E527E7E62622E2E323E12120E0C9
:10F40C00A06061A163A3A26266A6A767A56564A4B8
:10F41C006CACAD6DAF6F6EAEAA6A6BAB69A9A86828
:10F42C0078B8B979BB7B7ABABE7E7FBF7DBDBC7C18
:10F43C00B47475B577B7B67672B2B373B17170B088
:10F44C005090915193535292965657975595945478
:10F45C009C5C5D9D5F9F9E5E5A9A9B5B99595898E8
:10F46C00884849894B8B8A4A4E8E8F4F8D4D4C8CD8
:10F47C004484854587474686824243834181804048
:10FD76000117FF011E010134000118960139000127
:05FD86003500011C0026
:10FDBE00C208E47834F67838F6E51C6003B4FF0325
:04FDCE00751CFE2280
:0DFDF500C208E47834F67838F675189622C6
:09FE2600D2087F0A7E0002FE1BD7
:10FA3800E4F520D2DA7F0CFE12FE1BC2DAA2B092E5
:10FA480000D2DA7F087E0012FE1BC2DAA2B0920151
:10FA5800D2DA7F087E0012FE1BC2DAA2B09202D26E
:10FA6800DA7F087E0012FE1BC2DAA2B09203D2DA55
:10FA78007F087E0012FE1BC2DAA2B09204D2DA7F9F
:10FA8800087E0012FE1BC2DAA2B09205D2DA7F0805
:10FA98007E0012FE1BC2DAA2B09206D2DA7F087E7E
:10FAA8000012FE1BC2DAA2B09207D2DA7F087E00EB
:10FAB80012FE1B7834E6C394965007E606243AF8FB
:10FAC800A620C2097834E6FFB518057838760122F1
:10FAD800EF64077020783BE6FE64036004EEB4062A
:10FAE8000475180822EEB410087840E62409F518C1
:10FAF8002275189622EFB40104751AC822EFB403D0
:0BFB080009783BE6B4190375180622CB
:10FC75007833E6FF8F27752864D209C2B17F077EE6
:10FC85000012FE1BE4F529E5271392B1E527C313FE
:10FC9500F5277528127F077E0012FE1B0529E52929
:10FCA500C3940840E2D2B17F107E0012FE1BC20948
:01FCB500222C
:10FCF70012F7DD501312FE2612FE2F12F48C500558
:10FD070012F66A800302FDF512FDF5E517B4011737
:10FD1700E4FD7F107EEE12FD2FAD1C7F067EEF12F5
:08FD2700FD2F759F8080FE2274
:10F7DD007834E665186002C322783AE6FFF4600AD1
:10F7ED00EF651C6005EF6002C322783BE66419707B
:10F7FD007AFB7A00793A7D0412FC328E228F2378BF
:10F80D003EE6FE08E67C002400FFEC3EFEEF65239D
:10F81D007003EE65226002C322783DE6FF18E6FE16
:10F82D00C39F4004AD078002AD06EEC39F4004AFF9
:10F83D00068000E51CC39D4006E51CD39F4002C316
:10F84D0022AF0C7E0012FCED12FCB67C007D1E1268
:10F85D00FB3E8D25E4F524E524C39525500B7F64EF
:10F86D007E0012FE1B052480EED322783BE6FF645A
:10F87D0003600CEF64066007EF64106002C322782A
:10F88D003CE6FE08E67C002400FFEC3EFEEF640A39
:10F89D004E7042783BE6B4030C12FCB67C007D053D
:10F8AD0012FB3E8D1DE51D64016002C322AF0C7E6F
:10F8BD000012FCED12FCB67C007D1412FB3E8D2572
:10F8CD00E4F524E524C39525500B7F647E0012FEDC
:10F8DD001B052480EE7B007A00793AE51824FEFDA5
:10F8ED0012FC328E228F2374382518F8E6FE7439F7
:0AF8FD002518F8E67C002400FFEC5B
:0EF907003EFEEFB52306EEB52202D322C32248
:10F66A00E4F525783BE6B4061AE4F525743A25252F
:10F67A00F8E6FF12FC7912FE380525E525C3940841
:10F68A0040EA22783BE66403600302F77008E6FE6C
:10F69A0008E67C002400F523EC3EF522783FE6F5E7
:10F6AA0024783AE6FF12FC79783AE6FF12FDA87848
:10F6BA003BE6FF12FC79783BE6FF12FDA8E524251C
:10F6CA00E0FF12FC79E52425E0FF12FDA8E525C339
:10F6DA009524400302F763E4FF12FC79E4FF12FD6C
:10F6EA00A8E51EB47B167E00E5232525FFEE35220C
:10F6FA00FE7B007A00792612FE0F804E7E00E523FB
:10F70A002525FFEE3522FEC3EF940CEE9400500B34
:10F71A007B007A00792612FDD2802F7E00E5232510
:10F72A0025FFEE3522FEEF64204E700585BF268048
:10F73A0019EF642D4E7005851E26800EEF64304E3B
:10F74A0070058519268003752601AF2612FC79AF4C
:10F75A002612FDA8052502F6D712FC757836E6FFB3
:10F76A0012FC7902FE38783BE66410702CF5257499
:10F77A003A2525F8E6FF12FC79743A2525F8E6FFC2
:10F78A0012FDA80525E525C3940640E312FC757809
:10F79A0036E6FF12FC7902FE38783BE664197032CD
:03F7AA0018E6FF5F
:10F7AD0012FC79783AE6FF12FDA8783BE6FF12FCD1
:10F7BD0079783BE6FF12FDA8AF1C12FC79AF1C1245
:10F7CD00FDA812FC757836E6FF12FC7912FE382280
:10F48C00783BE664067064783DE6FFB406117E00B6
:10F49C00783FE6FD12FE02783FE6F51C02F5F078A7
:10F4AC003DE6B40A1CE51D6401600302F5F0783FEB
:10F4BC00E6FD7F067E0012FE02783FE6F51C02F5A3
:10F4CC00F0783DE6FFB410117E00783FE6FD12FEA9
:10F4DC0002783FE6F51702F5F0783DE6642D6003FF
:10F4EC0002F5F0783FE6F51E02F5F0783BE6641085
:10F4FC00600302F5F0783FE6F52A08E6FD783CE675
:10F50C00FCFE08E6F97A002400F525EA3EF5248C89
:10F51C00288929E52A6D7036F526F527C3E5279548
:10F52C002AE5269400506074412527F8E6F523E57A
:10F53C00252527FFE5243526FEAD2312FD2F40019E
:10F54C002212FE380527E52770D2052680CEE4F579
:10F55C0026F527C3E527952AE52694005029E527AB
:10F56C0025E02442F8E6F523E5252527FFE524359B
:10F57C0026FEAD2312FD2F40012212FE380527E591
:10F58C002770D0052680CC783906E664087055784B
:10F59C0035E675F002A42411FFE5F034EEFEE4FD2F
:10F5AC0012FD2F7835E675F002A42412FFE5F03435
:0FF5BC00EEFEE4FD12FD2F783506E675F002A491
:10F5CB002411FFE5F034EEFEAD2812FD2F7835E661
:10F5DB0075F002A42412FFE5F034EEFEAD2912FD06
:10F5EB002FE47839F6E517B47F0FE47839F67835E0
:10F5FB00F675177E7580FB8064E517B43F1CE4F548
:10F60B0022AF2212FD9012FE380522E522C3945A36
:10F61B0040EF75173E7580FB8043E517B4330B1233
:10F62B00FE3812FDE57517348033E517B41F26122B
:10F63B00FE387D1F7F107EEE12FD2F7DF07F117E39
:10F64B00EE12FD2F7DF07F127EEE12FD2F75171E31
:0FF65B007580FB8008E517B4010312FE38D32237
:09FE2F00783676FF783376FF2265
:10FDA8007833E66FFF90F28C937836667933F7EF05
:06FDB80090F38C93F6228B
:10FC32008B268A2789288D29752A00752BFF7DFF3F
:10FC4200AF291529EF6026AB260528E528AA2770DB
:10FC520002052714F912FB13652BFF90F28C936DAA
:10FC6200752A00F52BEF90F38C93FD80D3E52BFEE4
:03FC7200EDFF2281
:04FD8B004100000033
:06FD2F008E2B8F2C8D2DA0
:10FD350012FE3875F65575F6AA75F65575BF048524
:10FD45002DF6E52BF5F4852CF575F7807B007A000B
:10FD5500792EAF2CAE2B12FE0FE52EB52D02D32238
:01FD6500C3DA
:01FD6600227A
:10FD900075F65575F6AA75F65575BF04EF25E0F5AD
:08FDA000F4E4F5F575F7822289
:10FDE50075F65575F6AA75F65575BF0475F7832230
:0BFE0F008F828E83E49312FB2C7F0196
:01FE1A0022C5
:0DFE020074002FF582E43400F583EDF0224A
:10FDD20074002FF582E43400F583E012FB2C12FB51
:03FDE20013FF22EA
:01F0000020EF
:0300000002F20009
:0CF20000787FE4F6D8FD7581CF02F2475C
:10FB1300BB010689828A83E0225002E722BBFE02F0
:09FB2300E32289828A83E4932223
:10FB2C00BB010689828A83F0225002F722BBFE01B8
:02FB3C00F322B2
:10FB3E00C2D5EC30E709B2D5E4C39DFDE49CFCEEE2
:10FB4E0030E715B2D5E4C39FFFE49EFE12FB74C3EB
:10FB5E00E49DFDE49CFC800312FB7430D507C3E4E6
:06FB6E009FFFE49EFE2251
:10FCB600AC2FAD30AE31AF32780FEFA2E2EC20E6DA
:10FCC60001B35D5E5FF47004FCFDFEFFEF13FFEE13
:10FCD60013FEED13FDEC13FCD8E08C2F8D308E3126
:10FCE6008F32EE547FFE228E2F8F30E4F531F532BF
:01FCF60022EB
:10F20C0002FBC9E493A3F8E493A34003F68001F254
:10F21C0008DFF48029E493A3F85407240CC8C33303
:10F22C00C4540F4420C8834004F456800146F6DFD2
:10F23C00E4800B010204081020408090FD67E47EFE
:10F24C00019360BCA3FF543F30E509541FFEE493C7
:10F25C00A360010ECF54C025E060A840B8E493A38E
:10F26C00FAE493A3F8E493A3C8C582C8CAC583CAB9
:10F27C00F0A3C8C582C8CAC583CADFE9DEE780BE71
:01FD8F000073
:10FB7400BC000BBE0029EF8DF084FFADF022E4CC75
:10FB8400F875F008EF2FFFEE33FEEC33FCEE9DEC3E
:10FB9400984005FCEE9DFE0FD5F0E9E4CEFD22ED84
:10FBA400F8F5F0EE8420D21CFEADF075F008EF2FCE
:10FBB400FFED33FD4007985006D5F0F222C398FDBF
:05FBC4000FD5F0EA225C
:00000001FF
